:100000000C9458000C943F010C948A010C947500D8
:100010000C9475000C9475000C9475000C9475008C
:100020000C9475000C9475000C9475000C9475007C
:100030000C9475000C9475000C9475000C9475006C
:100040000C9475000C9475000C94D5010C947500FB
:100050000C9475000C9475000C9475000C9475004C
:100060000C9477000C947500C600E500CB00E50009
:10007000D600E500DB00E500E000E500EB00EB006A
:10008000EB00EB00EB00EB00EB00EB00EB00EB0018
:10009000D600E500DB00E5004546476566670020C1
:1000A0002B2D2E3031323334353637383968000055
:1000B00011241FBECFEFD8E0DEBFCDBF11E0A0E01E
:1000C000B1E0E4EEF1E102C005900D92A031B1077C
:1000D000D9F721E0A0E1B1E001C01D92A939B20732
:1000E000E1F70E94DE020C94F0080C9400001F92CD
:1000F0000F920FB60F9211248F939F93AF93BF93DC
:10010000EF93FF938091B900887F803879F048F4AD
:10011000803609F06BC085EC8093BC0010922301FF
:100120006DC0883A39F1883B29F160C08091230184
:10013000882341F08F3F09F050C08091BB0080932D
:1001400022014BC08091BB00809323018091230149
:10015000853019F481E08093190180912301873063
:1001600019F481E0809318018091230181508093DC
:1001700023012FC08091230190E0FC013197E831E9
:10018000F10548F5EC5CFF4F0C946B068091200163
:100190009091210104C080911E0190911F018093D4
:1001A0001401909315019093BB0013C080911C0122
:1001B00090911D01F4CF80911A0190911B01EFCF16
:1001C0008091160190911701EACF809114018093DC
:1001D000BB0085EC03C01092BB0085E88093BC0097
:1001E000809123018F5F8093230108C08091BC0020
:1001F0008B7E8093BC0085EC8093BC00FF91EF91D7
:10020000BF91AF919F918F910F900FBE0F901F9054
:10021000189593E890937A0080937C0080917C00FD
:10022000806480937C0080917A00806480937A005F
:1002300080917A0086FDFCCF8091780090917900C2
:1002400045E080E090E020917A00206420937A00DD
:1002500020917A0026FDFCCF209178003091790022
:10026000820F931F415079F720917A002F772093C6
:100270007A0065E070E00E943806CB0108951F9275
:100280000F920FB60F9211242F933F934F935F93CA
:100290006F937F938F939F93AF93BF93EF93FF934E
:1002A00080918400909185004A9B05C09093130132
:1002B000809312011EC02091120130911301BC01E4
:1002C000621B730B80E090E00E94470527EE3CE83C
:1002D00040E350E40E94D50520E030E040E05FE3D9
:1002E0000E94B7040E941B0570931D0160931C01BE
:1002F000E89AFF91EF91BF91AF919F918F917F917C
:100300006F915F914F913F912F910F900FBE0F9082
:100310001F9018951F920F920FB60F9211242F93D2
:100320003F934F935F936F937F938F939F93AF937D
:10033000BF93EF93FF9380918400909185004B9B36
:1003400005C090931101809310011EC020911001EF
:1003500030911101BC01621B730B80E090E00E94A0
:10036000470527EE3CE840E350E40E94D50520E035
:1003700030E040E05FE30E94B7040E941B057093E9
:100380001B0160931A01E99AFF91EF91BF91AF9120
:100390009F918F917F916F915F914F913F912F919D
:1003A0000F900FBE0F901F9018951F920F920FB6CF
:1003B0000F9211248F939F93EF93FF938091C0002E
:1003C00087FF17C0E0912601F09127018091C600B8
:1003D000808381E0EB38F80730F43196F093270101
:1003E000E093260106C088E291E090932701809374
:1003F0002601FF91EF919F918F910F900FBE0F906B
:100400001F9018959C01E1ECF0E080818861808369
:10041000808180688083E2ECF0E080818660808368
:1004200040E050E084E0220F331F441F551F8A959F
:10043000D1F760E074E284EF90E00E944C06DA01AC
:10044000C9010197A109B109892F9A2FAB2FBB27A9
:10045000A7FDBA958093C50021502093C40088E27F
:1004600091E090932501809324019093270180933C
:10047000260108952091C00025FFFCCFFC0180815A
:100480008093C6000895CF93DF931F92CDB7DEB758
:100490008983CE0101960E943A0280E090E00F909D
:1004A000DF91CF910895CF93DF93EC01CE01219698
:1004B000FC012081222319F00E943A02F7CFDF913C
:1004C000CF9108958091C00087FFFCCF8091C60036
:1004D00090E008950C9462026AE672E083E492E090
:1004E0000C949E06CF93DF93FC01E253FF4FA08153
:1004F000B181EC01C453DF4F28813981A217B307C2
:10050000B9F02091C00025FF13C02C912093C600A4
:1005100020813181AC0145535F4F2417350718F412
:100520002F5F3F4F03C09C0128593F4F31832083E9
:10053000E0912401F09125012091260130912701BD
:100540002E173F07C1F1DC01AC59BF4FCD91DC91B3
:100550001197208128836D917C9111979C012B52DA
:100560003F4FE9013881EB012881321307C09C011C
:100570002C523F4FE90148814F5F48839C012D5920
:100580003F4F6217730728F4EB012196CD93DC935C
:1005900002C08D939C93D1E0EB38FD0730F4319687
:1005A000F0932501E093240106C088E291E0909346
:1005B000250180932401DF91CF91089510922201AB
:1005C00080E895E20E9402020E946C0282E580931C
:1005D000BA008091BC008B7E8093BC0085EC809338
:1005E000BC001092800084E08093810085E08093BD
:1005F000690086E091E00E941B0783B7817F83BF7B
:100600007894C0E0D8E180912301833081F050F4E8
:10061000813089F580E00E94090190932101809347
:10062000200129C0893059F08F3FF1F024C081E0CA
:100630000E94090190931F0180931E011CC082E05B
:100640000E940901BC0180E090E00E94470528E477
:1006500031EE4AEB5FE30E94D5050E941B057093C3
:1006600017016093160107C080912201853A19F4A1
:10067000F894FE01099580911901882379F0109270
:10068000190110921D0110921C01529A5A9AF5E319
:10069000FA95F1F700005A985298E89A809118015B
:1006A000882379F01092180110921B0110921A0100
:1006B000539A5B9A85E38A95F1F700005B9853980B
:1006C000E99A83B7816083BF889583B78E7F83BFA4
:1006D0009ACF6F927F929F92AF92BF92CF92DF920A
:1006E000EF92FF920F931F93CF93DF93CDB7DEB7B7
:1006F0002C970FB6F894DEBF0FBECDBF8C017B01E7
:100700003A01FC0117821682838181FF19C1CE0153
:1007100001965C01F801D380F701D3FC2591D3FE4B
:1007200021917F01222309F407C1253249F4D3FC2A
:100730002591D3FE21917F01253211F0912C1BC010
:10074000B801822F90E00E94E90663013601E2CFF2
:10075000222309F4F1C0622F70E08FE990E02C872A
:100760000E9493062C85892B49F0F701D3FC259133
:10077000D3FE21917F0197FEEBCF0CC0233221F4F1
:10078000F92DF0619F2EF1CF2C3639F4292D2068F8
:10079000922EEBCF222309F4CFC0622F70E088E9BC
:1007A00090E02C870E9493062C85892B41F06301F1
:1007B000F4E0CF0ED11CB8018FE390E012C02336D5
:1007C00041F0233789F0233521F5F92DF1609F2E73
:1007D0000BC0630122E0C20ED11CB801F30180817D
:1007E00091810E94E906B2CF630122E0C20ED11CC2
:1007F000F30160807180F30190FC859190FE8191FE
:100800003F01882309F4A2CFB80190E00E94E906D5
:10081000F2CF243611F0293639F5630197FE09C06D
:10082000F4E0CF0ED11CF30160817181828193814C
:100830000AC0F2E0CF0ED11CF301608171818827DC
:1008400077FD8095982FF92DFF7E9F2E97FF09C089
:1008500090958095709561957F4F8F4F9F4FF06475
:100860009F2E2AE030E038C02037A1F040F4283530
:10087000D1F02F3609F060C028E030E019C02537EC
:1008800019F0283751F058C0292D2F7E922E2AE0DA
:1008900030E00EC0892D8061982E992D9462992E9A
:1008A00020E130E005C0E92DE4609E2E20E132E039
:1008B000630197FE09C0F4E0CF0ED11CF301608103
:1008C00071818281938108C0F2E0CF0ED11CF301C7
:1008D0006081718180E090E0A5010E944807782E38
:1008E0007A1896FE05C0B8018DE290E00E94E906F4
:1008F00094FE16C0FE01E70DF11D8081803381F06A
:10090000B80180E390E00E94E90692FE09C0292D1B
:100910002072822F90E0B801885A9F4F0E94E9060A
:100920007A94F501E70DF11D8081B80190E00E94F5
:10093000E9067110F5CF0ACFF8018681978102C0D0
:100940008FEF9FEF2C960FB6F894DEBF0FBECDBF92
:10095000DF91CF911F910F91FF90EF90DF90CF909B
:10096000BF90AF909F907F906F9008955058BB2795
:10097000AA270ED0E0C0D1D030F0D6D020F031F48C
:100980009F3F11F41EF4C6C00EF4E095E7FBBCC017
:10099000E92FE2D080F3BA1762077307840795073F
:1009A00018F071F49EF5FAC00EF4E0950B2EBA2FF4
:1009B000A02D0B01B90190010C01CA01A001112465
:1009C000FF27591B99F0593F50F4503E68F11A1611
:1009D000F040A22F232F342F4427585FF3CF4695A2
:1009E00037952795A795F0405395C9F77EF41F16C4
:1009F000BA0B620B730B840BBAF09150A1F0FF0F8E
:100A0000BB1F661F771F881FC2F70EC0BA0F621F79
:100A1000731F841F48F4879577956795B795F79569
:100A20009E3F08F0B3CF9395880F08F09927EE0FFB
:100A300097958795089598D088F09F5790F0B92F93
:100A40009927B751A0F0D1F0660F771F881F991F23
:100A50001AF0BA95C9F712C0B13081F09FD0B1E059
:100A600008959CC0672F782F8827B85F39F0B93F69
:100A7000CCF3869577956795B395D9F73EF4909525
:100A80008095709561957F4F8F4F9F4F0895E894A3
:100A900009C097FB3EF490958095709561957F4FC6
:100AA0008F4F9F4F9923A9F0F92F96E9BB27939574
:100AB000F695879577956795B795F111F8CFFAF484
:100AC000BB0F11F460FF1BC06F5F7F4F8F4F9F4FB5
:100AD00016C0882311F096E911C0772321F09EE813
:100AE000872F762F05C0662371F096E8862F70E079
:100AF00060E02AF09A95660F771F881FDAF7880F53
:100B00009695879597F9089597F99F6780E870E023
:100B100060E008959FEF80EC089500240A94161673
:100B2000170618060906089500240A9412161306DB
:100B3000140605060895092E0394000C11F4882369
:100B400052F0BB0F40F4BF2B11F460FF04C06F5F85
:100B50007F4F8F4F9F4F089557FD9058440F551F5B
:100B600059F05F3F71F04795880F97FB991F61F02F
:100B70009F3F79F087950895121613061406551FA6
:100B8000F2CF4695F1DF08C0161617061806991F12
:100B9000F1CF86957105610508940895E894BB2707
:100BA00066277727CB0197F908950BD0C4CFB5DF1F
:100BB00028F0BADF18F0952309F0A6CFABCF1124A7
:100BC000EECFCADFA0F3959FD1F3950F50E0551FEC
:100BD000629FF001729FBB27F00DB11D639FAA2792
:100BE000F00DB11DAA1F649F6627B00DA11D661FE1
:100BF000829F2227B00DA11D621F739FB00DA11D02
:100C0000621F839FA00D611D221F749F3327A00DBB
:100C1000611D231F849F600D211D822F762F6A2F57
:100C200011249F5750408AF0E1F088234AF0EE0FDC
:100C3000FF1FBB1F661F771F881F91505040A9F7E9
:100C40009E3F510570F060CFAACF5F3FECF3983E16
:100C5000DCF3869577956795B795F795E7959F5F50
:100C6000C1F7FE2B880F911D9695879597F90895EA
:100C7000AA1BBB1B51E107C0AA1FBB1FA617B707C2
:100C800010F0A61BB70B881F991F5A95A9F78095DE
:100C90009095BC01CD010895052E97FB1EF400949C
:100CA0000E94630657FD07D00E94710607FC03D01F
:100CB0004EF40C94630650954095309521953F4F26
:100CC0004F4F5F4F089590958095709561957F4F38
:100CD0008F4F9F4F0895EE0FFF1F0590F491E02D69
:100CE0000994A1E21A2EAA1BBB1BFD010DC0AA1F6D
:100CF000BB1FEE1FFF1FA217B307E407F50720F085
:100D0000A21BB30BE40BF50B661F771F881F991FFF
:100D10001A9469F760957095809590959B01AC0148
:100D2000BD01CF010895FC010590061621F00020B9
:100D3000D9F7C00108953197CF0108950F931F93FC
:100D4000CF93DF93EC018B01009731F461157105AE
:100D500019F480E090E038C06EE070E081E090E04F
:100D60000E94A607FC010097A1F380E88383011588
:100D7000110571F01387028781E8838380918F01C9
:100D800090919001892B21F4F0939001E0938F01D1
:100D90002097C9F0D187C087838182608383809147
:100DA000910190919201892B71F4F0939201E0935B
:100DB00091018091930190919401892B21F4F093FA
:100DC0009401E0939301CF01DF91CF911F910F9197
:100DD00008950F931F93CF93DF93182F092FEB01E3
:100DE0008B8181FD03C08FEF9FEF20C082FF10C079
:100DF0004E815F812C813D81421753077CF4E8814D
:100E0000F9819F012F5F3F4F39832883108306C0EC
:100E1000E885F985812F0995892B29F72E813F8156
:100E20002F5F3F4F3F832E83812F902FDF91CF91F4
:100E30001F910F9108950F931F93CF93DF93E0912C
:100E40009101F0919201238121FF1BC0EC0100E090
:100E500010E089916091910170919201DB011896E7
:100E6000ED91FC911997882331F00995892B89F32D
:100E70000FEF1FEFEECF8AE00995892B11F4C8011F
:100E800002C08FEF9FEFDF91CF911F910F910895D7
:100E9000FA01AA27283051F1203181F1E8946F93AB
:100EA0006E7F6E5F7F4F8F4F9F4FAF4FB1E03ED051
:100EB000B4E03CD0670F781F891F9A1FA11D680FEF
:100EC000791F8A1F911DA11D6A0F711D811D911D22
:100ED000A11D20D009F468943F912AE0269F112497
:100EE0003019305D3193DEF6CF010895462F4770FB
:100EF000405D4193B3E00FD0C9F7F6CF462F4F7056
:100F0000405D4A3318F0495D31FD4052419302D0B3
:100F1000A9F7EACFB4E0A695979587957795679559
:100F2000BA95C9F700976105710508959B01AC0159
:100F30000A2E06945795479537952795BA95C9F780
:100F4000620F731F841F951FA01D08950F931F9399
:100F5000CF93DF93869F8001879F100D969F100D82
:100F60001124C8010E94C207EC01009729F0A801D2
:100F700060E070E00E94E908CE01DF91CF911F91FF
:100F80000F910895CF93DF938230910510F482E0A2
:100F900090E0E0919701F091980120E030E0A0E02E
:100FA000B0E0309739F14081518148175907B8F0C6
:100FB0004817590771F482819381109729F013968D
:100FC0009C938E9312972CC09093980180939701D5
:100FD00027C02115310531F04217530718F0A90138
:100FE000DB0101C0EF019A01BD01DF010280F38145
:100FF000E02DD7CF21153105F9F0281B390B24300E
:10100000310580F48A819B816115710521F0FB0116
:101010009383828304C09093980180939701FE018B
:10102000329644C0FE01E20FF31F81939193225048
:101030003109398328833AC0209195013091960176
:10104000232B41F42091020130910301309396014A
:101050002093950120910001309101012115310566
:1010600041F42DB73EB74091040150910501241B76
:10107000350BE0919501F0919601E217F307A0F48A
:101080002E1B3F0B2817390778F0AC014E5F5F4FDE
:101090002417350748F04E0F5F1F50939601409379
:1010A00095018193919302C0E0E0F0E0CF01DF91E0
:1010B000CF910895CF93DF93009709F487C0FC0187
:1010C000329713821282C0919701D0919801209794
:1010D00081F420813181280F391F809195019091F1
:1010E00096018217930779F5F0939601E0939501A5
:1010F0006DC0DE0120E030E0AE17BF0750F412965D
:101100004D915C9113979D014115510509F1DA014B
:10111000F3CFB383A28340815181840F951F8A1737
:101120009B0771F48D919C911197840F951F0296E6
:101130009183808312968D919C91139793838283E0
:101140002115310529F4F0939801E09397013EC0F1
:10115000D9011396FC93EE9312974D915D91A40FD4
:10116000B51FEA17FB0779F480819181840F951FE1
:101170000296D90111969C938E9382819381139646
:101180009C938E931297E0E0F0E08A819B81009718
:1011900019F0FE01EC01F9CFCE01029628813981C8
:1011A000820F931F209195013091960128173907DE
:1011B00069F4309729F4109298011092970102C0B7
:1011C00013821282D0939601C0939501DF91CF9143
:1011D0000895DC0101C06D9341505040E0F708953F
:0411E000F894FFCFB1
:1011E4000000990120000D0A53746172740D00000F
:00000001FF
